:10000000523084000730FE001C30FF0011208000B9
:10001000840A0408703A03191528FF0A0319FE0A16
:1000200006287E088A007F088200831770308400CB
:100030007E301C208301242864008001840A040689
:100040000319003404061D2803108316031300301F
:1000500003180130850003100030031801308600BA
:1000600003108312031300300318013085000310BE
:1000700000300318013086003A2706250030F200D0
:100080000030F3004328720883120313A0002007F6
:10009000523E831384000008A100840A0008A200D5
:1000A000C625C830E127062503108312031300304C
:1000B00003180130A100003094250130F207031825
:1000C000F30A0030F3077308803A83120313A00089
:1000D00080302002031D6E280E307202031C71282E
:0600E000722843280028ED
:100A0C00013083120313860066256430E127080049
:100A1C0083120313A400240886003B250D30831297
:100A2C000313A5001A2D1A2D0130A502031D1F2D2D
:100A3C00202D192D0800A6000310003003180130DA
:100A4C00A700261C2A2D2B2D2F2D2508A8002808A1
:100A5C00A7070310A50D0310A60CA608031D372D20
:100A6C00382D272D27083A2D0800F9147908850010
:100A7C001130A600422D422D0130A602031D472D38
:100A8C00482D412D7915790885001130A7004F2D7F
:100A9C004F2D0130A702031D542D552D4E2DFB302B
:100AAC00A9002908F905790885001130A8005F2DE7
:100ABC005F2D0130A802031D642D652D5E2D0800ED
:100ACC00FD30A9002908F905790885001130A60028
:100ADC00702D702D0130A602031D752D762D6F2DF6
:100AEC007915790885001130A7007D2D7D2D0130F9
:100AFC00A702031D822D832D7C2DFB30A900290814
:100B0C00F905790885001130A8008D2D8D2D013047
:100B1C00A802031D922D932D8C2D0800A2000230EB
:100B2C00860066256430E127283083120313A50064
:100B3C002208212583120313A40021082407A200F4
:100B4C000310003003180130A100BF2D14308600B3
:100B5C006625213083120313A300B52DB52D01306A
:100B6C00A302031DBA2DBB2DB42D0130A400240803
:100B7C00A10722082102031CC42DC52DAC2D080091
:100B8C002208A601A6072108A501A5070B30A40081
:100B9C00743032260030FA000030FB00D52D7A0874
:100BAC00743E840000080E257A08013E743E8400D1
:100BBC008008031DE22DE32DE42DF92D0130FA07F9
:100BCC000318FB0A0030FB077B08803A83120313DF
:100BDC00A30080302302031DF52D04307A02031C80
:100BEC00F82DF92DD52D0800360835040319FF2DE5
:100BFC00002E302EB7010314B70D0F2E0130031049
:100C0C00B50DB60DFF3E031D052E0130B80038089A
:100C1C00B707B61F122E132E042E36083402031DEE
:100C2C00192E35083302031C1C2E1D2E232E3508BD
:100C3C00B3023608031CB403B40201300310B60C23
:100C4C00B50CFF3E031D242E0130B702031D2F2EC1
:100C5C00302E132E312E0800A9002530AA00EA2EC2
:100C6C002B08253A03193B2E3C2E472E2B08B0009F
:100C7C0029088400300880000130B0003008A90732
:100C8C00EA2E0310003003180130A800502EF72E66
:100C9C00622EEA2E00010138A4070001FF38240758
:100CAC000927AB00003A03194D2E643A03194E2E56
:100CBC000D3A03194E2E4F2E2A0884008313000878
:100CCC00AC00840A0008AD000230B0003008AA075E
:100CDC00AD1F712E722E7B2E0330B0003008A8048D
:100CEC00AC09AD09AC0A0319AD0AAB010314AB0D89
:100CFC007F2E2B08B0003007013EB2000927B1004F
:100D0C00B20A32080927B20032082D02031D902EB8
:100D1C0031082C020318932E942E952E9F2E013001
:100D2C00B0003008AB072B08053A031D9E2E9F2EF2
:100D3C007F2E280803390319A42EA52EAF2E2D3093
:100D4C00B00029088400300880000130B000300861
:100D5C00A9072B08A700E02E2708B0003007013E9A
:100D6C00B1000927B500B10A31080927B6002D08D2
:100D7C00B401B4072C08B301B307942783120313EF
:100D8C003408B401B4073308B301B3070A30B50013
:100D9C000030B600FA25831203133308303EAB0043
:100DAC002B08B00029088400300880000130B00006
:100DBC003008A907FF30B0003008A7072708FF3A12
:100DCC00031DE92EEA2EB22E00010138A407000102
:100DDC00FF3824070927AB00AB08031DF62EF72EAE
:100DEC00362E0310290884000030031801308000CF
:100DFC00FF2E0800FE00FE1F082F83137E1883179A
:100E0C00000808000408FE0007308A007E088207EC
:100E1C000034013400340A34003464340034E834CF
:100E2C000334103427342534643400349D34FF34B7
:100E3C00413400341734003454340034FF34FF345C
:100E4C00083400342D34003416340034403400346B
:100E5C00233400348834FF343034003421340034EB
:100E6C00F534FF344D34003438308600662532308A
:100E7C00E127383083120313860066252130831254
:100E8C000313A1004A2F4A2F0130A102031D4F2F3B
:100E9C00502F492F383086006625213083120313DA
:100EAC00A200592F592F0130A202031D5E2F5F2F74
:100EBC00582F383086006625213083120313A30087
:100ECC00682F682F0130A302031D6D2F6E2F672F23
:100EDC000130860066253230E1270D308312031372
:100EEC0086006625213083120313A4007E2F7E2FEB
:100EFC000130A402031D832F842F7D2F0630860022
:100F0C006625213083120313A5008D2F8D2F013000
:100F1C00A502031D922F932F8C2F08000030B800D0
:100F2C000030B9003608350403199D2F9E2FD92F98
:100F3C00B7010314B70DAD2F01300310B50DB60D6D
:100F4C00FF3E031DA32F0130BA003A08B707B61FA6
:100F5C00B02FB12FA22F01300310B80DB90DFF3EE9
:100F6C00031DB22F36083402031DBE2F3508330281
:100F7C00031CC12FC22FCC2F3508B3023608031C1B
:100F8C00B403B4020130B8040030B90401300310CA
:100F9C00B60CB50CFF3E031DCD2F0130B702031D5F
:100FAC00D82FD92FB12F3908B401B4073808B301A1
:100FBC00B307E02F080083120313A6000430A70028
:100FCC005330A800EA2FEA2F0130A802031DEF2F9F
:100FDC00F02FE92F0130A702031DF52FF62FE62F76
:0E0FEC000130A602031DFB2FFC2FE42F08008E
:02400E00693F08
:00000001FF
